:020000040000FA
:04080000E4EF04F02D
:1008100003B23DEF04F0F2B458EF04F09EB060EF85
:1008200004F09EB268EF04F0F2A81AEF04F0F2B2FE
:100830001CEF04F0C2EF04F0CD90F29207BC078EDB
:10084000078C9EA029EF04F00101463F29EF04F038
:10085000472B07AE34EF04F0CECF4EF1CFCF4FF1A0
:1008600046C150F147C151F1CF6ACE6A0101466BD2
:10087000476B9E90CD80C2EF04F00392030103EE1C
:1008800000F080517F0BE92604C0EFFF802B8151DF
:10089000805D700BD8A48B8200008051815D700B4D
:1008A000D8A48B9281518019D8B40790C2EF04F07C
:1008B000F2940101383FC2EF04F0392BC2EF04F08B
:1008C0009E900101463FC2EF04F0472BC2EF04F0B7
:1008D0009E92C3CF48F1C4CF49F1C28207B485EFDD
:1008E00004F03AC13EF13BC13FF13CC140F13DC192
:1008F00041F14EC152F14FC153F150C154F151C1B8
:1009000055F148C14AF149C14BF10201002FC2EF34
:1009100004F03C0E006FD57ED5BE32D0D6CF3AF172
:10092000D7CF3BF138C13CF1E86AE8CF3DF1010196
:1009300047A7A6EF04F0079C079E0101000E4E6F2B
:10094000600E4F6F3D0E506F080E516F01013ABFA0
:10095000B6EF04F03B67B6EF04F03C67B6EF04F087
:100960003D67B6EF04F0F288BBEF04F0F2984E6BEF
:100970004F6B506B516BD76AD66A0101386B396B7C
:10098000C2EF04F002C0E0FF005001C0D8FF100029
:10099000A6B2C8EF04F00CC0A9FF0BC0A8FFA69E2A
:1009A000A69CA684F29E550EA76EAA0EA76EA682DE
:1009B000F28EA694A6B2DAEF04F01200A96EA69EFB
:1009C000A69CA680A8501200076A0F010E0EC16EE9
:1009D000800EC06E030EC26E0F01896A110E926EF8
:1009E000080E8A6EF10E936E8B6A800E946EF18EF5
:1009F0000F01280ED56EF28AB00ECD6E9D800101DA
:100A00004E6B4F6B506B516B526B536B546B556B02
:100A1000566B576B586B596B079C079E760ECA6EC8
:100A20009D8202013C0E006FCC6A240EAC6E040164
:100A3000806B816B0F01900EAB6E0F019D8A0301DD
:100A4000806B816BA26B8B9207900001F28EF28C0F
:100A500007B086EF0CF08B740301805181197F0B76
:100A6000D8B486EF0CF013EE00F081517F0BE12635
:100A7000812BE7CFE8FFE00BD8B486EF0CF023EE34
:100A800082F0A2511F0BD926E7CFDFFFA22BDF5048
:100A9000780AD8A486EF0CF007808251720AD8B485
:100AA00008EF07F08251630AD8B446EF09F082518B
:100AB000690AD8B47BEF05F082517A0AD8B48EEF78
:100AC00006F07BEF09F0040114EE00F080517F0B7B
:100AD000E12682C4E7FF802B12000D0E826F63ECCB
:100AE00005F00A0E826F63EC05F01200040E826FAF
:100AF00063EC05F012000401690E826F63EC05F0EF
:100B000004012C0E826F63EC05F00101030E006FEF
:100B1000000E016F000E026F000E036F15EC0FF058
:100B200020C182F40401300E822763EC05F021C15C
:100B300082F40401300E822763EC05F022C182F4B6
:100B40000401300E822763EC05F023C182F4040116
:100B5000300E822763EC05F024C182F40401300ECC
:100B6000822763EC05F025C182F40401300E822750
:100B700063EC05F026C182F40401300E822763EC99
:100B800005F027C182F40401300E822763EC05F0E2
:100B900004012C0E826F63EC05F00101030E006F5F
:100BA000000E016F000E026F000E036F15EC0FF0C8
:100BB00020C182F40401300E822763EC05F021C1CC
:100BC00082F40401300E822763EC05F022C182F426
:100BD0000401300E822763EC05F023C182F4040186
:100BE000300E822763EC05F024C182F40401300E3C
:100BF000822763EC05F025C182F40401300E8227C0
:100C000063EC05F026C182F40401300E822763EC08
:100C100005F027C182F40401300E822763EC05F051
:100C200004012C0E826F63EC05F001010B0E006FC6
:100C3000000E016F000E026F000E036F15EC0FF037
:100C400020C182F40401300E822763EC05F021C13B
:100C500082F40401300E822763EC05F022C182F495
:100C60000401300E822763EC05F023C182F40401F5
:100C7000300E822763EC05F024C182F40401300EAB
:100C8000822763EC05F025C182F40401300E82272F
:100C900063EC05F026C182F40401300E822763EC78
:100CA00005F027C182F40401300E822763EC05F0C1
:100CB00004012C0E826F63EC05F0200EF86EF76ACB
:100CC000F66A04010900F5CF82F463EC05F009002F
:100CD000F5CF82F463EC05F00900F5CF82F463EC04
:100CE00005F00900F5CF82F463EC05F00900F5CFBB
:100CF00082F463EC05F00900F5CF82F463EC05F0B3
:100D00000900F5CF82F463EC05F00900F5CF82F419
:100D100063EC05F06DEC05F07BEF09F08351630A9D
:100D2000D8A47BEF09F08451610AD8A47BEF09F0C5
:100D300085516C0AD8A47BEF09F08651410A42E044
:100D40008651440A1BE08651420AD8B4F5EF06F0FA
:100D50008651350AD8B404EF0BF08651360AD8B460
:100D600058EF0BF08651370AD8B4C0EF0BF086511C
:100D7000380AD8B41EEF0CF07BEF09F00798079AF9
:100D800004017A0E826F63EC05F00401780E826F25
:100D900063EC05F00401640E826F63EC05F081A83A
:100DA000D9EF06F00401550E826F63EC05F0DEEF1B
:100DB00006F004014C0E826F63EC05F06DEC05F05B
:100DC0007BEF09F00788079A04017A0E826F63ECC3
:100DD00005F00401410E826F63EC05F00401610E21
:100DE000826F63EC05F0CFEF06F00798078A0401E5
:100DF0007A0E826F63EC05F00401420E826F63ECA1
:100E000005F00401610E826F63EC05F0CFEF06F090
:100E10000401720E826F63EC05F004012C0E826FE8
:100E200063EC05F0078452C156F153C157F154C128
:100E300058F155C159F13EC142F13FC143F140C1A2
:100E400044F141C145F14AC14CF14BC14DF1079408
:100E50000101620E046F010E056F000E066F000E99
:100E6000076F56C100F157C101F158C102F159C1D4
:100E700003F17BEC0EF003BF85EF07F00E0EDEEC06
:100E800004F0E8CF0CF10F0EDEEC04F0E8CF0DF12A
:100E9000100EDEEC04F0E8CF0EF1110EDEEC04F0E3
:100EA000E8CF0FF1C4EC0DF056C104F157C105F1C4
:100EB00058C106F159C107F17BEC0EF0078288ECAE
:100EC0000DF0C4EC0DF0079288EC0DF056C100F166
:100ED00057C101F158C102F159C103F1079288ECE1
:100EE0000DF0CC0E046FE00E056F870E066F050E39
:100EF000076F7BEC0EF000C10CF101C10DF102C1D6
:100F00000EF103C10FF1BEEF07F00101800E006F7B
:100F10001A0E016F060E026F000E036F42C104F13C
:100F200043C105F144C106F145C107F17BEC0EF068
:100F300003AF9FEF07F072EC0FF0D1EF07F00E0E4A
:100F4000DEEC04F0E8CF0CF10F0EDEEC04F0E8CF9D
:100F50000DF1100EDEEC04F0E8CF0EF1110EDEEC18
:100F600004F0E8CF0FF142C100F143C101F144C1E7
:100F700002F145C103F1078288EC0DF00CC100F1CC
:100F80000DC101F10EC102F10FC103F10101000E0B
:100F9000046F000E056F010E066F000E076FA9ECBF
:100FA0000EF015EC0FF01D67DBEF07F00401200ECB
:100FB000826FDEEF07F004012D0E826F63EC05F007
:100FC00024C182F40401300E822763EC05F025C1B0
:100FD00082F40401300E822763EC05F004012E0E2A
:100FE000826F63EC05F026C182F40401300E822783
:100FF00063EC05F027C182F40401300E822763EC14
:1010000005F004016D0E826F63EC05F004012C0EF7
:10101000826F63EC05F042C100F143C101F144C1AC
:1010200002F145C103F1010115EC0FF01EC182F47C
:101030000401300E822763EC05F01FC182F4040125
:10104000300E822763EC05F020C182F40401300EDB
:10105000822763EC05F021C182F40401300E82275F
:1010600063EC05F022C182F40401300E822763ECA8
:1010700005F023C182F40401300E822763EC05F0F1
:1010800024C182F40401300E822763EC05F025C1EF
:1010900082F40401300E822763EC05F026C182F44D
:1010A0000401300E822763EC05F027C182F40401AD
:1010B000300E822763EC05F00401480E826F63EC6A
:1010C00005F004017A0E826F63EC05F004012C0E2A
:1010D000826F63EC05F056C100F157C101F158C1B0
:1010E00002F159C103F1010115EC0FF01EC182F4A8
:1010F0000401300E822763EC05F01FC182F4040165
:10110000300E822763EC05F020C182F40401300E1A
:10111000822763EC05F021C182F40401300E82279E
:1011200063EC05F022C182F40401300E822763ECE7
:1011300005F023C182F40401300E822763EC05F030
:1011400024C182F40401300E822763EC05F025C12E
:1011500082F40401300E822763EC05F026C182F48C
:101160000401300E822763EC05F027C182F40401EC
:10117000300E822763EC05F00401630E826F63EC8E
:1011800005F004012C0E826F63EC05F056C100F1EE
:1011900057C101F158C102F159C103F101010A0E11
:1011A000046F000E056F000E066F000E076F8AECCD
:1011B0000EF0000E046F120E056F000E066F000E8B
:1011C000076FA9EC0EF015EC0FF01EC182F40401BC
:1011D000300E822763EC05F01FC182F40401300E4B
:1011E000822763EC05F020C182F40401300E8227CF
:1011F00063EC05F021C182F40401300E822763EC18
:1012000005F022C182F40401300E822763EC05F060
:1012100023C182F40401300E822763EC05F024C15F
:1012200082F40401300E822763EC05F004012E0ED7
:10123000826F63EC05F025C182F40401300E822731
:1012400063EC05F026C182F40401300E822763ECC2
:1012500005F027C182F40401300E822763EC05F00B
:101260000401730E826F63EC05F004012C0E826F93
:1012700063EC05F072EC0FF04CC100F14DC101F1CF
:10128000A4EC0AF06DEC05F07BEF09F00401630EAD
:10129000826F63EC05F004012C0E826F63EC05F0A5
:1012A00080EC09F004012C0E826F63EC05F0F3EC86
:1012B00009F004012C0E826F63EC05F06FEC0AF06C
:1012C00004012C0E826F63EC05F00101F80E006F33
:1012D000CD0E016F660E026F030E036F95EC09F0E1
:1012E00004012C0E826F63EC05F085EC0AF06DECC6
:1012F00005F07BEF09F00301A26B079086EF0CF07D
:10130000D8900E0EDEEC04F0E8CF00F10F0EDEEC0C
:1013100004F0E8CF01F1100EDEEC04F0E8CF02F1AA
:10132000110EDEEC04F0E8CF03F10101000E046FB2
:10133000000E056F010E066F000E076FA9EC0EF090
:1013400015EC0FF01EC182F40401300E822763EC0D
:1013500005F01FC182F40401300E822763EC05F012
:1013600020C182F40401300E822763EC05F021C114
:1013700082F40401300E822763EC05F022C182F46E
:101380000401300E822763EC05F023C182F40401CE
:10139000300E822763EC05F024C182F40401300E84
:1013A000822763EC05F025C182F40401300E822708
:1013B00063EC05F004012E0E826F63EC05F026C18C
:1013C00082F40401300E822763EC05F027C182F419
:1013D0000401300E822763EC05F004016D0E826F6C
:1013E00063EC05F01200120EDEEC04F0E8CF00F121
:1013F000130EDEEC04F0E8CF01F1140EDEEC04F085
:10140000E8CF02F1150EDEEC04F0E8CF03F10101A4
:101410000A0E046F000E056F000E066F000E076FB8
:101420008AEC0EF0000E046F120E056F000E066FB0
:10143000000E076FA9EC0EF015EC0FF01EC182F440
:101440000401300E822763EC05F01FC182F4040111
:10145000300E822763EC05F020C182F40401300EC7
:10146000822763EC05F021C182F40401300E82274B
:1014700063EC05F022C182F40401300E822763EC94
:1014800005F023C182F40401300E822763EC05F0DD
:1014900024C182F40401300E822763EC05F00401BC
:1014A0002E0E826F63EC05F025C182F40401300E2C
:1014B000822763EC05F026C182F40401300E8227F6
:1014C00063EC05F027C182F40401300E822763EC3F
:1014D00005F00401730E826F63EC05F012000A0E32
:1014E000DEEC04F0E8CF00F10B0EDEEC04F0E8CF08
:1014F00001F10C0EDEEC04F0E8CF02F10D0EDEEC93
:1015000004F0E8CF03F1A4EF0AF0060EDEEC04F0DD
:10151000E8CF00F1070EDEEC04F0E8CF01F1080E91
:10152000DEEC04F0E8CF02F1090EDEEC04F0E8CFC7
:1015300003F1A4EF0AF0010172EC0FF007844AC135
:1015400000F14BC101F107940101E80E046F800E18
:10155000056F000E066F000E076F8AEC0EF0000E8E
:10156000046F040E056F000E066F000E076FA9ECE6
:101570000EF0880E046F130E056F000E066F000E3E
:10158000076F7BEC0EF00A0E046F000E056F000E65
:10159000066F000E076FA9EC0EF015EC0FF00101BD
:1015A0001D67D8EF0AF00401200E826FDBEF0AF00E
:1015B00004012D0E826F63EC05F024C182F4040156
:1015C000300E822763EC05F025C182F40401300E51
:1015D000822763EC05F026C182F40401300E8227D5
:1015E00063EC05F004012E0E826F63EC05F027C159
:1015F00082F40401300E822763EC05F00401430EEF
:10160000826F63EC05F0120087C31EF188C31FF1DF
:1016100089C320F18AC321F18BC322F18CC323F14A
:101620008DC324F18EC325F190C326F191C327F118
:101630000101BFEC0FF037EC0FF00101000E046F59
:10164000000E056F010E066F000E076F8AEC0EF09C
:101650000E0E0C6E00C10BF0C8EC04F00F0E0C6EF9
:1016600001C10BF0C8EC04F0100E0C6E02C10BF0BF
:10167000C8EC04F0110E0C6E03C10BF0C8EC04F0C2
:1016800004017A0E826F63EC05F004012C0E826F68
:1016900063EC05F00401350E826F63EC05F0040184
:1016A0002C0E826F63EC05F080EC09F0DEEF06F0A3
:1016B00087C31EF188C31FF189C320F18AC321F1BA
:1016C0008BC322F18CC323F18DC324F18EC325F18A
:1016D00090C326F191C327F10101BFEC0FF037EC65
:1016E0000FF0880E046F130E056F000E066F000ECC
:1016F000076F7FEC0EF0000E046F040E056F000EF6
:10170000066F000E076F8AEC0EF00101E80E046F01
:10171000800E056F000E066F000E076FA9EC0EF02D
:101720000A0E0C6E00C10BF0C8EC04F00B0E0C6E30
:1017300001C10BF0C8EC04F00C0E0C6E02C10BF0F2
:10174000C8EC04F00D0E0C6E03C10BF0C8EC04F0F5
:1017500004017A0E826F63EC05F004012C0E826F97
:1017600063EC05F00401360E826F63EC05F00401B2
:101770002C0E826F63EC05F06FEC0AF0DEEF06F0E2
:1017800087C31EF188C31FF189C320F18AC321F1E9
:101790008BC322F18CC323F18DC324F18FC325F1B8
:1017A00090C326F191C327F10101BFEC0FF037EC94
:1017B0000FF0000E046F120E056F000E066F000E84
:1017C000076F8AEC0EF001010A0E046F000E056F20
:1017D000000E066F000E076FA9EC0EF0120E0C6ED5
:1017E00000C10BF0C8EC04F0130E0C6E01C10BF03D
:1017F000C8EC04F0140E0C6E02C10BF0C8EC04F03F
:10180000150E0C6E03C10BF0C8EC04F004017A0E47
:10181000826F63EC05F004012C0E826F63EC05F01F
:101820000401370E826F63EC05F004012C0E826F09
:1018300063EC05F0F3EC09F0DEEF06F087C31EF170
:1018400088C31FF189C320F18AC321F18BC322F120
:101850008CC323F18DC324F18EC325F190C326F1EF
:1018600091C327F10101BFEC0FF037EC0FF0880EA8
:10187000046F130E056F000E066F000E076F7FECEE
:101880000EF0000E046F040E056F000E066F000EC2
:10189000076F8AEC0EF00101E80E046F800E056FF1
:1018A000000E066F000E076FA9EC0EF0060E0C6E10
:1018B00000C10BF0C8EC04F0070E0C6E01C10BF078
:1018C000C8EC04F0080E0C6E02C10BF0C8EC04F07A
:1018D000090E0C6E03C10BF0C8EC04F004017A0E83
:1018E000826F63EC05F004012C0E826F63EC05F04F
:1018F0000401380E826F63EC05F004012C0E826F38
:1019000063EC05F085EC0AF0DEEF06F081A844EF09
:101910000DF007A8FDEF0CF00101800E006F1A0E0C
:10192000016F060E026F000E036F3EC104F13FC14E
:1019300005F140C106F141C107F17BEC0EF003BF98
:1019400044EF0DF082EC0DF03EC100F13FC101F11A
:1019500040C102F141C103F1078288EC0DF00CC1D6
:1019600004F10DC105F10EC106F10FC107F1F80E2A
:10197000006FCD0E016F660E026F030E036F7BECDE
:101980000EF00E0E0C6E00C10BF0C8EC04F00F0E42
:101990000C6E01C10BF0C8EC04F0100E0C6E02C10D
:1019A0000BF0C8EC04F0110E0C6E03C10BF0C8EC88
:1019B00004F00784010172EC0FF04AC100F14BC141
:1019C00001F107940A0E0C6E00C10BF0C8EC04F094
:1019D0000B0E0C6E01C10BF0C8EC04F00C0E0C6E7B
:1019E00002C10BF0C8EC04F00D0E0C6E03C10BF03D
:1019F000C8EC04F0079844EF0DF007AA44EF0DF08F
:101A00000784010172EC0FF04AC100F14BC101F1F2
:101A10000794060E0C6E00C10BF0C8EC04F0070E24
:101A20000C6E01C10BF0C8EC04F0080E0C6E02C184
:101A30000BF0C8EC04F0090E0C6E03C10BF0C8ECFF
:101A400004F0078452C100F153C101F154C102F105
:101A500055C103F10794120E0C6E00C10BF0C8ECD7
:101A600004F0130E0C6E01C10BF0C8EC04F0140E60
:101A70000C6E02C10BF0C8EC04F0150E0C6E03C125
:101A80000BF0C8EC04F0079A0401805181197F0B18
:101A90000BE09EA809D014EE00F081517F0BE126E7
:101AA000E750812B0F01AD6E28EF05F00CC100F15E
:101AB0000DC101F10EC102F10FC103F1000E046F5F
:101AC000000E056F010E066F000E076FA9EC0EF0F9
:101AD0001DA181EF0DF01451D8B481EF0DF00CC1B0
:101AE00000F10DC101F10EC102F10FC103F1000EB1
:101AF000046F000E056F0A0E066F000E076FA9EC4B
:101B00000EF0120001010C6B0D6B0E6B0F6B1200CF
:101B10000101005305E1015303E1025301E1002BF0
:101B20004BEC0EF072EC0FF02C51006F2D51016F49
:101B3000420E046F4B0E056F000E066F000E076F0E
:101B40008AEC0EF000C104F101C105F102C106F1F9
:101B500003C107F10CC100F10DC101F10EC102F189
:101B60000FC103F107B2B9EF0DF07FEC0EF0BBEF40
:101B70000DF07BEC0EF000C10CF101C10DF102C1C2
:101B80000EF103C10FF1120072EC0FF04CC100F125
:101B90004DC101F1060EDEEC04F0E8CF04F1070EB2
:101BA000DEEC04F0E8CF05F1080EDEEC04F0E8CF3F
:101BB00006F1090EDEEC04F0E8CF07F17BEC0EF045
:101BC00000C118F101C119F102C11AF103C11BF1E1
:101BD000290E046F000E056F000E066F000E076FD2
:101BE0008AEC0EF0EE0E046F430E056F000E066FCA
:101BF000000E076F7FEC0EF018C104F119C105F15A
:101C00001AC106F11BC107F18AEC0EF000C110F1F8
:101C100001C111F102C112F103C113F1120EDEEC88
:101C200004F0E8CF04F1130EDEEC04F0E8CF05F188
:101C3000140EDEEC04F0E8CF06F1150EDEEC04F035
:101C4000E8CF07F10D0E006F000E016F000E026F5E
:101C5000000E036F8AEC0EF0180E046F000E056F75
:101C6000000E066F000E076FA9EC0EF010C104F114
:101C700011C105F112C106F113C107F17FEC0EF09D
:101C80006A0E046F2A0E056F000E066F000E076FB6
:101C90007BEC0EF01200BF0EFA6E200E2D6F2C6B37
:101CA000D8900037013702370337D8B05CEF0EF019
:101CB0002D2F51EF0EF02C072D070353D8B412002F
:101CC0000331070B8009326F03390F0B010F2C6FA3
:101CD00080EC5FF0336F2C0580EC5FF0335D335F99
:101CE0002C6B3233D8B02C272C3332A971EF0EF085
:101CF00033512C27120097EC0FF0D8B0120003518B
:101D00000719286F5AEC0FF0D8900751031928AF24
:101D1000800F1200286B7EEC0FF0D8A094EC0FF02F
:101D2000D8B0120069EC0FF072EC0FF01F0E296FA3
:101D3000AAEC0FF00B35D8B05AEC0FF0D8A0033551
:101D4000D8B01200292F98EF0EF028B181EC0FF0D7
:101D50001200286B04510511061107110008D8A0C4
:101D60007EEC0FF0D8A094EC0FF0D8B01200086B06
:101D7000096B0A6B0B6BAAEC0FF01F0E296FAAEC14
:101D80000FF007510B5DD8A4D2EF0EF006510A5D9B
:101D9000D8A4D2EF0EF00551095DD8A4D2EF0EF011
:101DA0000451085DD8A0E5EF0EF00451085F05511D
:101DB000D8A0053D095F0651D8A0063D0A5F07512E
:101DC000D8A0073D0B5FD8900081292FBFEF0EF000
:101DD00028B181EC0FF0286B7EEC0FF0D890AEECC0
:101DE0000FF007510B5DD8A402EF0FF006510A5D0A
:101DF000D8A402EF0FF00551095DD8A402EF0FF04F
:101E00000451085DD8A011EF0FF0003F11EF0FF063
:101E1000013F11EF0FF0023F11EF0FF0032BD8B489
:101E2000120028B181EC0FF012000101286B7EEC4A
:101E30000FF0D8B01200B3EC0FF0200E296F00376E
:101E400001370237033711EE27F00A0E2A6FE73603
:101E50000A0EE75CD8B0E76EE5522A2F27EF0FF0A5
:101E6000292F1FEF0FF028B11D81D890120001011A
:101E70000A0E286F200E296F11EE1DF028512A6FCF
:101E80000A0ED890E652D8B0E726E7322A2F42EF62
:101E90000FF00333023301330033292F3CEF0FF0EF
:101EA000E750FF0FD8A00335D8B012001DB181EC68
:101EB0000FF01200045100270551D8B0053D01274D
:101EC0000651D8B0063D02270751D8B0073D032779
:101ED00012000051086F0151096F02510A6F03513E
:101EE0000B6F12000101006B016B026B036B1200A0
:101EF0000101046B056B066B076B12000335D8A05C
:101F000012000351800B001F011F021F031F003F1F
:101F100091EF0FF0013F91EF0FF0023F91EF0FF0C3
:101F2000032B282B032512000735D8A012000751D8
:101F3000800B041F051F061F071F043FA7EF0FF0AC
:101F4000053FA7EF0FF0063FA7EF0FF0072B282B59
:101F500007251200003701370237033708370937E2
:101F60000A370B3712001D6B1E6B1F6B206B216B2A
:101F7000226B236B246B256B266B276B12001E5183
:101F80000F0B1E6F1F510F0B1F6F20510F0B206F78
:101F900021510F0B216F22510F0B226F23510F0B79
:101FA000236F24510F0B246F25510F0B256F2651E2
:0C1FB0000F0B266F27510F0B276F12003C
:10BF0000E844F926000C160C2B0C3F0C520C640C68
:10BF1000760C860C960CA50CB30CC10CCF0CDC0C6B
:06BF2000E80CF40C000C1B
:00000001FF
